:020000040000FA
:02000000F029E5
:080008000000F500030EF600F4
:10001000031383120A08F7008A010408F800831208
:1000200003138C1E252883120313320884008312C5
:10003000031347238313831203138000B10AB20A08
:100040003208453A35300319B20083120313831383
:100050007808840077088A00760E8300F50E750E06
:02006000090095
:1000800082070A340D343E347734583458345934A6
:1000900020347734723469347434653420347634DF
:1000A00061346C3475346534203459342034403430
:1000B000203461346434643472346534733473349A
:1000C0002034583458340A340D3420342034203449
:1000D00020342034203472346534743475347234EE
:1000E0006E34733420347734313420346F346E34CA
:1000F0002034733475346334633465347334733447
:100100000A340D343E347434203420342034203406
:1001100044344534533454345234553443345434D1
:100120004934563445342034733465346C34663481
:100130002D3474346534733474340A340D342034FB
:100140002034203420342034203465346D34693434
:1001500074347334203427344F344B3427342034F0
:100160006F346E34203473347534633463346534DF
:100170007334733420346F3472342034273446346B
:10018000413449344C34273420346F346E342034B5
:100190006634613469346C347534723465340A34CD
:1001A0000D340A340D34003483120313B00083126B
:1001B00003130C1ED7288312031330088312031372
:1001C0003F2B831203133108003E0319E3288313E6
:1001D000330884000008B400B103B30A3308453A79
:1001E00035300319B3003408831203138313080056
:1002000082070A340D340A340D34533465347234A1
:10021000453445342034763431342E3432340A3483
:100220000D3443346F346D346D3461346E34643462
:1002300073343A340A340D343E34723458345834FA
:1002400020342034723465346134643420343134E1
:1002500020346234793474346534203440342034AA
:1002600061346434643472346534733473342034E8
:1002700058345834203428343234203462347934B9
:100280007434653473342C3420346C3469347434ED
:1002900074346C3465342D3465346E3464346934AC
:1002A00061346E3429340A340D342034203420343F
:1002B000203420342034723465347434753472340C
:1002C0006E347334203472343134593420346F3402
:1002D0006E3420347334753463346334653473346A
:1002E000733420342834593420346934733420343E
:1002F000623469346E346134723479342034723447
:100300006534733475346C34743420346234793425
:100310007434653429340A340D343E34523458343C
:1003200058342034203472346534613464342034D9
:1003300058345834203428343234203462347934F8
:100340007434653473342C3420346C34693474342C
:1003500074346C3465342D3465346E3464346934EB
:1003600061346E3429342034623479347434653421
:1003700073342C34203473347434613472347434F0
:1003800069346E346734203440342034613464344A
:1003900064347234203430340A340D342034203440
:1003A000203420342034203472346534743475346D
:1003B00072346E34733420346134203464347534D0
:1003C0006D34703420346F346634203461346C34CE
:1003D0006C342034623479347434653473340034CA
:1003E0008B01031383168E1581170030850036307C
:1003F0008600831207309F008501860183138312D4
:100400000313B0222523831203133530B200B30047
:10041000B101831603138C16831203130B17831277
:1004200003138B17831203135523C50101308A0070
:1004300045080021003E0319202AD420C50F162AA2
:10044000C50100308A0045084020003E03192B2AD0
:10045000D420C50F212A4730D4206F30D4200A3051
:10046000D4200D30D420E1203E3A031D332AA023AE
:10047000332AA5000830A4008612A50D031886169D
:10048000000083160313061683120313061E462A62
:10049000831603130612831203130612A40B3C2ABD
:1004A000831603138616061683120313061E562A96
:1004B00000000111861A0115831603138612061215
:1004C000831203130612861208008316031386167E
:1004D000831203130830A4000612831603130612B6
:1004E000831203130310A501A50D8316031306162B
:1004F00083120313061E7A2A861A251406128316FF
:100500000313061283120313A40B742A2508080090
:1005100086128316031386128312031300008316B8
:100520000313061683120313000006128316031327
:10053000061283120313080086168316031386120D
:10054000831203130000831603130616831203138A
:100550000000061283160313061283120313080009
:10056000FA301923FA3019230800A1007008A200FC
:100570007108A300DC22A03039220119BA2A22080E
:1005800039222308392221083922F3220800A20047
:100590007008A300DC22A03039220119CA2A2208DF
:1005A000392223083922DC22A13039226522A10018
:1005B0009C22F322210808008316031306168616D0
:1005C00083120313061A861EE22A83160313861269
:1005D000831203138612000083160313061283127C
:1005E0000313061208008612000083160313061672
:1005F000831203138616080083169B001C141A0826
:1006000083120800F0009C18022B71089B007008F0
:100610009A0003108B1B031483161C158B13553083
:100620009D00AA309D009C141C11831203188B1787
:100630000800A7000430A800FB30A900A90B1E2B5E
:10064000A80B1C2BA70B1A2B080083160615861463
:1006500018150C30990098131813981618121810C2
:100660008312181398121816181118109817FA30C8
:1006700019231A081A081A0800309900080083166E
:10068000981C402B83120C1E3F2B990008009818D1
:100690004F2B8C1E472B1A0818194B2B08001812C9
:1006A0001A081A081A081816472B08007230D420A6
:1006B000E120F000E120C722F2003130D42072089E
:1006C000D42008005230D420E120F200E120F300D1
:1006D000F0010030C722D420F20B712BF30B712BE9
:1006E0000800D322D4206C2B7430D420FF30F300C8
:1006F000F0017308F100B5222E30D4207308F00009
:100700000030C7227306031D8C2BF30B782B4F3060
:10071000D4204B30D42008004630D4204130D4209F
:100720004930D4204C30D42008007730D420E12048
:10073000F100E120F000E120B5223130D4200800A2
:10074000E120F200723A0319562B7208523A03194B
:10075000622B7208773A0319952B7208743A0319C1
:04076000742B0800EE
:02400E00503F21
:00000001FF
